:100000000C9446000C9463000C9463000C94630001
:100010000C9463000C9463000C9463000C946300D4
:100020000C9463000C9463000C9463000C946300C4
:100030000C9463000C9463000C9463000C946300B4
:100040000C9435020C9463000C9463000C946300D0
:100050000C9463000C9463000C9463000C94630094
:100060000C9463000C9463000C9463000C94630084
:100070000C9463000C9463000C9463000C94630074
:100080000C9463000C9497000C94630011241FBE21
:10009000CFEFD0E1DEBFCDBF11E0A0E0B1E0E2E202
:1000A000F6E000E00BBF02C007900D92A230B1074E
:1000B000D9F712E0A2E0B1E001C01D92AF35B1075F
:1000C000E1F70C94C0000C940000CF93DF93FC0187
:1000D0009C012C5F3F4F848180931D01C82FDD2739
:1000E000F90142815381DE01AA0FBB1FAB5FBE4FF6
:1000F0008D919C9111978417950741F4FE01E95E5B
:10010000FE4F9081F9018181981761F04D935C93C6
:10011000DE01A95EBE4FF90181818C93CF5EDE4F77
:1001200081E0888382E090E0DF91CF9108951F9273
:100130000F920FB60F9211242F933F934F935F931B
:100140006F937F938F939F93AF93BF93EF93FF939F
:100150000E945C01E4E7F0E0808180688083FF9189
:10016000EF91BF91AF919F918F917F916F915F912F
:100170004F913F912F910F900FBE0F901F901895A8
:10018000CFEFD0E1DEBFCDBF0E946A028091640054
:1001900080618093640085E690E00E946E01882370
:1001A00031F480916500806180936500FFCF789481
:1001B0000E946A0283E00E9496028091000180936F
:1001C0001D011EC0E22FFF27EE0FFF1FEB5FFE4F4A
:1001D0008CED95E0918380836CED75E0822F0E9419
:1001E000BC0290911D01E92FFF27DF01A95EBE4FE0
:1001F0001C92EF5EFE4F81E080839F5F90931D0114
:1002000020911D01809101018217E0F6809100018B
:100210002CC0A92FBB27FD01E95EFE4F80818823FA
:1002200009F1FD01EF5EFE4F8081815080838823BC
:1002300031F06CED75E0892F0E94BC0213C0AA0F4B
:10024000BB1FAB5FBE4F6D917C91892F0E94BC029A
:10025000E0911D01FF27DF01A95EBE4F8C91EF5E8B
:10026000FE4F808380911D018F5F80931D019091CF
:100270001D0180910101891760F6C0E0D0E00E9465
:100280005E02809102019091030169E170E00E9499
:10029000FD02892B31F48091650090E189278093DC
:1002A00065002196C230D10551F7B0CFE0911E0113
:1002B000F0911F0109950895E0912001F09121012D
:1002C00089E292E0099599270895E0912201F09141
:1002D0002301BC0184E291E009950895CF93DF9357
:1002E000EC0184E090EFA1E0B0E0ABBFFC018791AE
:1002F00096918750904B09F05BC086E090EFA1E0AB
:10030000B0E0ABBFFC0187919691AC0166277727DF
:10031000440F551F661F771F6BBFFA018791969197
:10032000039708F445C04E5F5F4F6F4F7F4F26E045
:1003300030E08EE191E00E94F3029091720086E33A
:10034000E9E2F2E0282F11922A95E9F78093290239
:1003500081E080932A0280932B0210922D0210924A
:100360002C02D0932F02C0932E0281B38C7F81BBCD
:1003700082B38C7F82BB80E2809370008091740096
:10038000846080937400809174008068809374000E
:100390008091740081608093740080917400806407
:1003A000809374009E7F9093720081E090E002C081
:1003B00080E090E0DF91CF910895009731F0A0EABE
:1003C000BFE01197F1F70197D1F70895009731F049
:1003D000A4E0B0E01197F1F70197D1F70895282F25
:1003E00009C084E690E0A0EABFE01197F1F7019719
:1003F000D1F721502223A9F70895282F09C081E0C1
:1004000090E0A0EABFE01197F1F70197D1F72150F2
:100410002223A9F70895282F09C08AE090E0A0EAD6
:10042000BFE01197F1F70197D1F721502223A9F7E7
:100430000895282F09C08AE090E0A4E0B0E0119769
:10044000F1F70197D1F721502223A9F70895282F1A
:1004500009C084E690E0A4E0B0E01197F1F70197BD
:10046000D1F721502223A9F708951F920F920FB6BA
:100470000F9211248F939F93809104018F5F80933B
:1004800004018A3058F01092040180910201909189
:1004900003010196909303018093020186E082BFDD
:1004A0009F918F910F900FBE0F901F90189584E031
:1004B00083BF12BE81E087BF789408952091020126
:1004C00030910301809102019091030182179307FB
:1004D000C9F308959FEF9BBB1ABA98BB80E187BB15
:1004E00095BB14BA92BB11BA93B912B810926200BC
:1004F000109261009093650088E18093640010BEC3
:100500001092900089E189B91BB888E98AB98EE018
:100510008093950087EC86B980E487B986B1877CA3
:1005200011F03699FECF0E9457020895813071F480
:1005300080E49CE997BD86BD1DBC1CBC8AEA8FBDCA
:100540008AE18EBD87B3806E87BB0895833099F4AE
:1005500080E49CE990938100809380001092890050
:10056000109288008AEA80938B008AE180938A0047
:1005700082B1886382B90895660F771F8230A1F037
:10058000833028F4882351F0813009F50AC0843083
:10059000A9F0843070F08530D1F415C07BBD6ABD00
:1005A000089579BD68BD08957093790060937800CF
:1005B0000895709387006093860008957093850076
:1005C000609384000895709383006093820008957F
:1005D00097B1907C9062982B97B9369A3699FECF56
:1005E00085B1992708956BBFFA01DC0102C007901D
:1005F0000D9221503040D8F70895AA1BBB1B51E142
:1006000007C0AA1FBB1FA617B70710F0A61BB70B82
:10061000881F991F5A95A9F780959095BC01CD0127
:0206200008953B
:020622000305CE
:00000001FF
